:1000000015EF00F0EA6A060EE96EEF500DE0060EFD
:10001000016E006A002EFED7012EFBD77B0E006E0C
:10002000002EFED7EF2EF3D7000CF86AD09EEA6AB6
:10003000E96AC150C00B0F09C16E070EB46EC15002
:10004000C00B0F09C16EC090C092C094C09EC28008
:100050009698C69A949E93809392010EC66E000E57
:10006000C76ED190800ED56ECD6A000ECA6E000E9E
:10007000CB6E9484BD6AB76AB66A070EB46E9250AE
:10008000926E100E006E002EFED70000B450A19CA0
:10009000B56A929A899A040E056EFA0E066EB2DF60
:1000A000052EFBD7929A898A040E056EFA0E066E0B
:0A00B000A9DF052EFBD7EDD70300F2
:020000040030CA
:0E00000025CC390E0087A1000FC00FE00F4085
:00000001FF
